:020000040800F2
:2000000000080020DD000008E5000008E700000800000000000000000000000000000000F7
:20002000000000000000000000000000E90000080000000000000000EB000008ED000008E7
:20004000EF000008EF000008EF000008EF000008EF000008EF000008EF000008EF000008E8
:2000600000000000EF000008EF000008EF000008EF000008EF00000800000000EF000008B6
:2000800000000000000000000000000000000000EF0000080000000000000000EF00000872
:2000A00000000000EF0000080000000000000000EF000008EF00000800000000000000005B
:2000C0000548854600F02AFBC046C04600F03CF800480047410700080008002004488047A9
:2000E00004480047FEE7FEE7FEE7FEE7FEE7FEE771130008C100000830B50B46014600201D
:200100002022012409E00D46D5409D4205D31D469540491B2546954040191546521E002D43
:20012000F1DC30BD03460B439B0703D009E008C9121F08C0042AFAD203E00B780370401C17
:20014000491C521EF9D2704770B5054C054D03E0206800198047241DAC42F9D170BD00000F
:200160003C35000840350008F0B507460846584087B0C00F049048000E4659004008490889
:20018000BC1A884105D2384631461E4617460B4602465800400810434CD0300D0390400576
:2001A0005900400D490D0590401A0290402872DA18030121000B09050843019004980092AE
:2001C000002805D0019952420020884100920190029840210A1A0199009800F0D7F905468C
:2001E0000C466B4607CB00F0F2F9C0197141039A0E0D0023D71756401A467A40164344D0DE
:20020000049A002A2DD0029A012A039A15DC1205C01A914101263605001C7141D20F059E4D
:20022000D2070093019202962A46234600F0EFF907B0F0BD38463146FAE71605224A0F4660
:20024000B218C01AB74101210905001C4F4100187F41114618187941E20F10436D1964419E
:2002600013E0E2076D0815436408C2071443039A01261205C01A91413605001C7141CE07E4
:20028000400830434908C01851412A46234600F0B1F9CDE7FFE7049801224000C117121AD8
:2002A00000238B4104983146C417381AA141EEE730B40124E407634030BC55E730B4012490
:2002C000E407614030BC4FE70000E0FFF0B51FB488B00B990998002448400999C00F490036
:2002E00049080991C0070B990090490049080B9109990898A64608431CD00B990A980843EC
:2003000018D0099801244000420D4800410D099824050003000B204309900B980003000B85
:2003200020430B9050181C494018002201901446104605E0002001460DB0F0BD032801DA7B
:20034000034600E003239C46C11A0AAE0AE05F0008ADED5B4F00F75B7D430027AA187C418C
:20036000491C5B1E6145F2DD410004AB5A522104120C0A43240C401C0828DFDB019802905D
:200380000099704601910090059B049A0799069800F03DF9D0E700000DFCFFFFF0B50C4695
:2003A0005C4085B0E40FE40703944C000026640859009446490802460296224321D06246B7
:2003C0000A431ED06200570D4A000E032303550D012402462C492405781B1B0B360B4018DC
:2003E00023432643614600901C46501AB44103D30098401C009002E0921800985B410028F4
:2004000003DA0020014605B0F0BD0020012109050746864611E064461D46141BB54106D3D1
:200420006546521BB341744607430C43A646CD0740084908284392185B4105460D43EAD1FD
:200440001046184313D06046194650407140084306D06046101AB34106D20122002306E0D9
:2004600000220123DB0702E00122D2435310009874460105381C6141029C039D0019694188
:2004800000F0B8F8BFE70000FD03000070B54B005B0803430BD04B005C0D00263346654228
:2004A000B341D417AD1AA34102DB0020014670BD12053018514170BD0EB50549029100215E
:2004C00000910A460B46019100F0A1F803B000BD330400000EB5054A029200220092134675
:2004E000019200F094F803B000BD0000330400004A0009030123090B1B051943094B10B523
:20050000520D9A4201DA002010BD064B34339A4203DC9A1A00F04AF810BD03495118884035
:2005200010BD0000FF030000CDFBFFFFF0B51FB40646002082B005464024019100901BE044
:20054000019922460F46304600F030F8049A059B801A994110D310461946224600F016F806
:20056000361A8F410197224601200021009F00F00DF838184D4100902046641E0028DFDC4C
:20058000019B00982946324607B0F0BD10B5202A04DB0146203A9140002010BD914020237B
:2005A0009C1A0346E3401943904010BD10B5202A04DB0846203AD040002110BD0B46D34028
:2005C000D0402024A21A91400843194610BD10B5202A06DBCB170846203A1041C1170B43D2
:2005E00006E00B461341D0402024A21A91400843194610BD10B5002B08DA0024401C614124
:2006000092185B411A4301D14008400010BDF0B51FB482B005460C0003D0084601F04EFAB5
:2006200002E001F04BFA20300246009021462846FFF7ACFF049B059A04460F461843114378
:20064000084314D0184610431BD0009840210A1A18460599FFF7AAFF05460E46009A059940
:200660000498FFF793FF084305D0012004E02046394607B0F0BD0020C11705430E432C43E8
:20068000374300990E986305401A7905E40A00220C43FD0A0A3002D500200146E9E70105AD
:2006A000101969410C9C0D9D00196941FFF7A2FFDFE700004A0009030123090B1B051943EB
:2006C0000A4B10B5520D9A4202DA0020014610BD064B34339A4203DC9A1AFFF767FF10BD65
:2006E000034BD218FFF752FF10BD0000FF030000CDFBFFFF10B5002904DB0124E407404287
:200700008C412146002B04DB1C460123DB075242A341994200D1904210BD0000064C0125F8
:20072000064E05E0E36807CC2B430C3C98471034B442F7D3FFF7C8FC1C3500083C3500083D
:2007400010B5C046C04602F00FF910BD0B680022002B6FD0F8B5012425460B6895402B4012
:2007600069D04E68022E01D0122E14D1D608B600371800973F6A5607BC46F70E0F26BE46A4
:20078000BE406746B743BC460E697746BE4067463E43009F3E624E68012E05D0022E03D056
:2007A000112E01D0122E16D186680327B4465600B646B7406646BE43B446CF687646B74016
:2007C0006646374387604668AE430D79ED06ED0F954035434560076856000325B540AC4632
:2007E000AF430D79AD07AD0FB5403D430560C7686546AF438D68B5403D43C5604D68ED003A
:2008000040D5244D6E6B26436E639508224CAD002F19BC6895072E0F0F25B540AC43052500
:200820002D07A84201D100250CE01C4DA84203D1012507E02CE025E0194DA84201D1022529
:2008400000E00625B5402543BD60164C25684E689D43F60300D51D43256065684E689D4378
:20086000B60300D51D436560A5684E689D43F60200D51D43A560E5684E689D43B60200D580
:200880001D43E5600B68521CD34000D063E7F8BD7047000000100240000001400004005052
:2008A00000080050000401400148006870470000E0000020002801D10120704770B50546F1
:2008C00004462035687D0026002803D12E752046C046C046022068752068016849084900D3
:2008E00001600F2160680906884321680861206882680121C9038A438260A068002807D0BD
:20090000E268012A01D021218902084321688860E068022802D121688002486020684168DF
:200920000C4A11434160616920690843A169090208432168C860216AE069084321680860AD
:200940002068026801210A430260A6636975002070BD00000080000202480168491C0160A5
:2009600070470000E000002010B506480168022211430160032000F007F8C046C04600202D
:2009800010BD00000020024070B52248416B042529434163416A29434162416AA9434162C0
:2009A00000F09EFC1D4C1C482060681FE0601D481B490068FFF7A0FB401E60600020206118
:2009C000A060204600F07DFB0021204600F09EFB0421204600F09AFB2068426A12490A6030
:2009E00009687D22D200891881631049142000F0D3FB01220E49100508602068C168114349
:200A0000C1602068C1682943C160204600F072FB002070BD00100240000801403C0100206F
:200A200040420F00E4000020D0000020992E000800E100E0F8B505465E480F460068C0077F
:200A4000C00FB8420AD25B49086840084000384308600868C007C00FB8427DD12878564CE2
:200A6000800705D5E068F0218843A9680843E0602878C00765D06868022822D0002824D0B1
:200A80002168032825D049076DD5E168890889000143E160FFF708FF6968064602291BD003
:200AA00003292AD00029E16838D00907890F012947D0FFF7F9FE811B404881423CD90320A1
:200AC000F8BD216889034ED5DFE7216889054AD5DBE7890147D5D8E7E1680907890F0229EA
:200AE0002FD0FFF7E1FE811B34488142E7D8E0680007800F0228F4D123E0E1680907890FC7
:200B000003291ED0FFF7D0FE811B2C488142D6D8E0680007800F0328F4D112E00907890F0E
:200B20000FD0FFF7C1FE811B24488142C7D8E0680007800FF5D104E0E0680007800F012828
:200B4000B7D11C480168C907C90FB9420DD3016849084900394300E005E001600068C007E9
:200B6000C00FB84201D00120F8BD2878400706D5E068072109028843E9680843E060287881
:200B8000000707D5E0680721C90288432969C9000843E06000F038F8E168094A0906090FA3
:200BA000515CC840074908600320FFF7EDFE0020F8BD0000002002400010024088130000A0
:200BC00074320008E4000020044805490068C968044A4905490F515CC8407047E4000020CC
:200BE000001002408D320008044805490068C968044A8904490F515CC8407047E400002006
:200C0000001002408D32000810B51D4A5068D3680004410F0C2003401A4805D0042B06D09D
:200C2000082B0BD00C2B0BD0491C884010BD1068C00601D5144810BD144810BD144810BD0B
:200C4000D068D1688002134B000F185C0902D368890F01242404491C234207D11268D206A1
:200C600009D5094A5043FFF747FA10BD084A5043FFF742FA10BD054A5043FFF73DFA10BDEC
:200C8000001002400080000000093D000024F40000127A0084320008F8B504460078C007A4
:200CA00052D0FD4EF0680007800F022807D0F0680007800F032809D1F068C00306D5306857
:200CC000800341D56068002875D03DE0012062680004824203D131680143316014E0052318
:200CE00001211B0489049A42326805D18243326032680A433260EEE7824332603268024002
:200D00000092306888433060606800280ED0FFF7CBFD05463068800316D4FFF7C5FD401B5F
:200D2000C8287DD830688003F7D50DE0FFF7BCFD05463068800307D5FFF7B6FD401BC828B5
:200D40006ED830688003F7D42078800745D5D24EF0681F270007800F3F02012807D0F06841
:200D60000007800F032809D1F068C00306D43068400719D5E06801281DD115E0E168092050
:200D8000002919D0326882430A433260FFF78CFD05463068400707D4FFF786FD401B022881
:200DA0003ED830684007F7D570682169B84309020843706011E0C0E0316881433160FFF77A
:200DC00073FD05463068400707D5FFF76DFD401B022825D830684007F7D42078C0065CD582
:200DE000AD4EF068AD4F0007800F23D0A069002840D03068B11508433060FFF755FD05460E
:200E00003068800507D4FFF74FFD401B022807D830688005F7D57068216AB843084300E0C2
:200E2000ACE070607068217F0002000A09060843706032E03068800502D5A06900287CD025
:200E40007068216AB843084370607068217F0002000A090608437060FFF7D6FEF168904A6E
:200E60000906090F515CC8408E4908600320FFF78BFD12E03168FF20013081433160FFF790
:200E800013FD05463068800507D5FFF70DFD401B022873D830688005F7D42078824D0007D8
:200EA00026D560690028286911D0012108432861FFF7FAFC06462869800719D4FFF7F4FCBB
:200EC000801B02285AD828698007F7D510E0400840002861FFF7E8FC06462869800707D51C
:200EE000FFF7E2FC801B022848D828698007F7D4207840077ED50020074600906648806B8E
:200F0000C00006D46448816B0204114381630120009066480068C00519D464480068FF21B4
:200F200001310843614908600127FFF7BDFC06465E480068C0050AD400E0C0E0FFF7B4FC28
:200F4000801B642879D859480068C005F4D5A168C81FF93813D001208002002915D00522A6
:200F60001202914211D12A6981108A432A612A6902432A612869084328610EE05DE02869A8
:200F8000FF2101310843286107E02969FF22013291432961296981432961A068002810D010
:200FA000FFF782FC2969064689051AD4404DFFF77BFC801BA84240D83B4800698005F6D590
:200FC0000FE0FFF771FC29690646890509D5384DFFF76AFC801BA8422FD83348006980059F
:200FE000F6D4002F04D03148026881158A430260009800E006E0002804D02748816B0204C1
:2010000091438163606A002857D0234DE9680907890F032953D001273F06022828680ED042
:20102000B8432860FFF740FC04462868800144D5FFF73AFC001B02283CD90320F8BDB8432E
:201040002860FFF731FC06462868800107D5FFF72BFC801B0228F0D828688001F7D4216B9A
:20106000E06AEA680843A16AFD231B049A4311430843E860286838432860FFF715FC044697
:201080002868800119D4FFF70FFC001B0228D4D828688001F7D510E00010024000E0000061
:2010A00074320008E400002040100240007000408813000028688001BAD40020F8BD01200C
:2010C000F8BD002801D10120704770B5054604462035687D002803D128752046C046C0468A
:2010E00002206875211D206800F0B6F901206875002070BD0222014620314A7502681368E1
:2011000001200343136048750020704710B40124224603688A40196A91431962196A114332
:201120001962006801682143016010BC00207047002801D10120704770B5054604466035DA
:20114000687A002803D128722046C046C0462420687220680168490849000160204600F045
:201160002FFA606A002802D0204600F097F9206841680922D20291434160206881682A223A
:201180009143816020680168012211430160204600F0EAF970BD0000F3B50B4D81B0AC6826
:2011A0000F46A8680121C906884207D1214686003446C0222046FEF7B5FFAE6001988000B8
:2011C0000019076403B0F0BD00ED00E021490A68520701D50020704710B58A6B92B001235C
:2011E0001B071A438A631C490A680323DB029A43CB14D2180A60232100915901002813D05F
:2012000005200004019002200990032080040B900120800500240C9003940A916846FFF7DB
:201220003BFD00280FD101E00191ECE70F200D9003200E900F941094012111940DA8FFF7E2
:20124000F9FB002802D0002012B010BD012012B010BD0000001002400070004038B500242E
:201260001349002808D0012810D0022817D011A0C046C046204638BD0524C86A2407012237
:201280001043C862C86A10400090F3E7124CCA6A02200243CA62C96A01400091EAE70F4C8F
:2012A000CA6A04200243CA62C96A01400091E1E70010024050696E6D6170206572726F7297
:2012C0003A2077726F6E6720706F7274206E756D6265722E0000000000040050000800501F
:2012E00070B51C4DE9680C2001401B481B4C05D0042909D0082909D00C2912D069680904FE
:20130000490F491C884002E0154800E015482060E86815490006000F085C2168C14021601A
:2013200070BDE868E9688002104A000F105C0902EA68890F01231B04491C1A4204D1084A68
:201340005043FEF7D9FEE2E7064A5043FEF7D4FEDDE700000010024000800000E400002021
:201360000024F40000127A00743200088432000870B5324C92B02068A11508432060E06827
:201380002F490840E06020682E4908402060A06840084000A06020680126B604B04320601A
:2013A000E068FD2109048843E060002525612649E0038860264925480860FFF7D5FA0120A0
:2013C000FFF704FF00282FD1FFF700FF00282BD1A06B21040843A0631E4801680322D2028D
:2013E0009143C2148918016023200090012003901020049002200990400501950C900B9623
:201400000A956846FFF748FC00280CD10F200D9003200E900F951095012111950DA8FFF7F7
:2014200009FB002800D0FEE7616A042001436162616A8143616212B070BD00000010024042
:201440000C40FF88F6FFF6FE00ED00E000127A00E40000200070004030B4026801239B07AF
:201460000D4C984201D0A04203D17025AA434D682A43984201D0A04204D103231B029A438C
:20148000CB681A4302608A68C262096881620121416130BC704700000008014010B4818C6F
:2014A000C90707D001684A6801235B049A43836A1A434A60818C890707D501684A6801235E
:2014C0001B049A43C36A1A434A60818C490707D501684A6801239B049A43036B1A434A6073
:2014E000818C090707D501684A680123DB039A43436B1A434A60818CC90607D50268916829
:2015000001231B039943836B19439160818C890607D501688A6801235B039A43C36B1A43B5
:201520008A60818C490612D503685A6801210905046C8A4322435A60026C8A4207D1026849
:20154000516803235B059943436C19435160818C090607D501684A680123DB04806C9A43D5
:2015600002434A6010BC704770B5044600680068124D000708D501212B460022490520460E
:2015800000F0ACF900280CD12068006840070AD501212B4600228905204600F09FF9002842
:2015A00001D0032070BD0021204660300172E166202141728172002070BD0000F0550000C0
:2015C000F8B504462669A368E7693343666900203E4325683343B54A2E680146B44F3E40E4
:2015E0001E432E6025686B6803263603B343E66833436B602568A369954201D0266A33436E
:20160000AE680B273F02BE431E43AE60A94E2568A94BB5420AD1DB680C26334016D0042B8A
:2016200039D0082B35D00C2B10D10EE095420DD1DE6803239B021E4008D001239B02F61A9E
:2016400029D0F61A25D09E4200D108209B4B954274D10026002820D0022840D004286FD0CE
:2016600008283BD164682046FEF726FF07460091F107600808437108FEF72CFF0022904BC3
:20168000FEF772FD3A46009BFEF788FEFEF730FF09E10220DAE70420D8E767683846FEF73A
:2016A0000BFF05460091F107780808437108FEF711FF06460F46FFF787FAFEF7FDFE0822D1
:2016C000FEF7E4FE32463B46FEF74EFD2A46009BFEF764FEFEF70CFF2168C860F8BD1868B2
:2016E0006468C006204614D5FEF7E6FE07460091F107600808437108FEF7ECFE0022714B71
:20170000FEF732FD3A46009BFEF748FEFEF7F0FEC9E0FEF7D1FE07460091F1076008084376
:201720007108FEF7D7FE0022674BFEF71DFD3A46009BFEF733FEFEF7DBFEB4E022E0FFE7F8
:2017400067683846FEF7B8FE05460091F107780808437108FEF7BEFE06460F46FFF754FAE3
:20176000FEF7AAFE0822FEF791FE32463B46FEF7FBFC2A46009BFEF711FEFEF7B9FE2168F5
:20178000C860F8BD0122E669D20396424BD1092841D202007A44127992189744040E183CB7
:2017A0002A3C3C3C3400FFF70FFA616840004A088018FEF7A1FC81B22DE0FFF715FA616885
:2017C00040004A088018FEF797FC81B223E018686168C00606D53D4A48088018FEF78CFC4B
:2017E00081B218E03A4A48088018FEF785FC81B211E0FFF709FA616840004A088018FEF7D7
:201800007BFC81B207E061680122480812048018FEF772FC81B20A0908071201400F2168AA
:201820001043C860F8BD0928FCD201007944097949188F44050F1904290404043300F1E794
:20184000FFF7C2F961684A088018FEF755FC2168C860F8BDFFF7C8F961684A088018FEF719
:201860004BFC2168C860F8BD18686168C00605D5184A48088018FEF73FFC14E0164A4808B4
:201880008018FEF739FC0EE0FFF7BEF961684A088018FEF731FC2168C860F8BD6168480897
:2018A0008018FEF729FCE860F8BD000000480040F369FFEF0044004040100240001002403F
:2018C000000060418084CE418084EE4100127A000048E80100093D000024F400F8B51D46F6
:2018E00017460E460446FEF7DFFF394627460090603720680029C169304602D088432CD01D
:2019000054E0884352D0681C21D0002D05D0FEF7CBFF0099401AA84219D92068026880210E
:201920008A43026021680A68202082430A6021680A68C3009A430A6021688A6852085200E2
:201940008A607872B872002038720320F8BD2068C16930468843D6D128E0681C21D0002DA3
:2019600005D0FEF7A1FF0099401AA84219D9206801688022914301602068026820218A4366
:20198000026020680268CB009A430260206882685208520082607972B972002038720320E6
:2019A000F8BD2068C16930468843D6D00020F8BD10B5044600F02AFDE06801F06AFA606081
:2019C0000020A06000F068FD10BD10B5044600F01DFD2068002805D1E06801F05AFA6060D9
:2019E0000120206000F058FD10BD70B5044600F00DFD00F00BFD20680025002804D0E068E2
:201A000001F047FA6168451A00F046FDA0682C1800F042FD204670BD70B5002505604560D7
:201A20000446856000F064FDE06000F0EFFCE06801F02FFAA560606000F02EFD204670BD36
:201A400010B5144600F02AFFA04201D0012010BD002010BDCAB2012110B50A43002319468E
:201A600000F0E2FE10BD10B500F000FF10BD000010B5044600202060204600F05FFE054998
:201A8000204600F0E5FD0121204600F0E2FE204610BD0000A086010037B514460846064B77
:201AA0006A46214600F010F904466946002000F0A7FC20463EBD0000012400082021020C8D
:201AC00001D010211046020A01D010460839020901D01046091F820801D01046891E42083E
:201AE00001D0881E7047081A704702E008C8121F08C1002AFAD170477047002001E001C10D
:201B0000121F002AFBD1704710B50E480024046044608460C4600621046100F041FD0A488C
:201B20000521046044608460C460046100F026FD0648FFF771FF09220A210548FFF798FF13
:201B400010BD000004010020180100202C010020CC000020F0B51FB486B00998089A030D20
:201B60000021024314D05148514A1818504305141198012810981AD0281A401C00264D4F47
:201B80004D49009601910490002812DA444211E01198012449A3012801D11098C143069869
:201BA000119A84600360C26041600BB0F0BD4042E4E70446210500203F4A001C5141039160
:201BC000029012E0E00707D032463B4601990098FEF77CFB0191009032463B46104619465C
:201BE000FEF774FB06460F466410002CEAD10498039B0028029A0999089806DAFEF766FB0F
:201C0000019B009AFEF762FB05E0FEF7C7FB019B009AFEF7C3FB04460E460022284BFEF78F
:201C200069FD03D80020C043014607E00022254B20463146FEF798FAFEF73CFD102409E0D1
:201C4000002C0ADB0A220023FEF770FC079B30321A55641E02460A43F2D11122641C079B21
:201C6000121B1C19119B012B03D0012308430ED10AE0084304D0112010900020119077E710
:201C80001098151A6D1E0BE01098824202DD00236D1C03E0824201DA00236D1E002BEED0E7
:201CA000069811998260C16030C07EE701FCFFFF104D0000000014400000F03F3000000079
:201CC0000000F0430000E03FFFB597B00646002518E2252877D100242746FD49049400E068
:201CE0000443761C32780120203A90400842F7D130782A280ED0022230780146303909297E
:201D000016D804990A235943303940181443761C0490F1E7189802C804911890002904DA9B
:201D20000120400304434842049002200443761C30782E2814D1042004437078761C2A28C5
:201D400009D11898761C80C8189009E00A214F43303FC719761C3078014630390929F5D998
:201D600030786C2810D006DC4C281AD068280ED06A2817D104E0742813D07A2812D110E047
:201D80000120400504430CE00121090501E0032109050C437178814203D101200005241836
:201DA000761C761C3078119066280BD013DC58287DD009DC00287BD04528F6D04628F4D0D4
:201DC00047281AD1A5E118E0632835D0642870D0652812D19DE170286CD008DC6728F1D0D9
:201DE00069287BD06E280DD06F2806D1BAE073282ED0752871D0782859D01A9A199990470F
:201E00006D1C7EE16002400F022809D003280DD00428189801680DD00D60001D189070E179
:201E20001898EA1701680D604A60F6E7189801680D80F2E70D70F0E718986A460178117265
:201E4000001D18900020507202A80090012005E0189802C8189000200091C04361070DD57B
:201E6000002101E00199491C0191B94212DA8142F8DB009A515C0029F4D10BE0002101E030
:201E80000199491C01918142FADB019A0099895C0029F5D1019904981A9B471A21463846E0
:201EA000199A00F097FA0199401945180BE04FE02CE113E04EE0009800990078491C0091B7
:201EC0001A9A199990470198401E0190401CF2D1214638461A9B199A10E137E00A2000217E
:201EE000009001916002410F022907D0189A01CA1892C2179446032908D00AE01898C01DB7
:201F0000C108C90005C91891944607E000B2C2179446042902D140B2C1178C46002261462D
:201F2000944506DA0A460021404291418C462D2102E0210504D52B216A461173012103E09D
:201F4000E10701D02021F7E7029155E00A200AE0102008E0102000900021042004430191D7
:201F6000082703E008200021019100906002410F022907D0189A01CA1892002294460329E1
:201F800008D008E01898C01DC108C90005C91891944603E080B2042900D1C0B200210291D8
:201FA000210729D51199702906D0009A1021019B4A401A4305D00EE040216A46117301211A
:201FC00008E06146014306D030216A4611731199517302210291009A0821019B4A401A4369
:201FE0000AD16146014301D1610705D530216A46117301217F1E02911199582904D035A15B
:020000040800F2
:202000000E910DA90D910DE037A1F9E76146019B009AFEF78BFA0E9B8C469B5C0D9A521E48
:202020000D92137061460143F0D10D9805A9081A20300190600703D501200004844300E071
:2020400001270198874201DD381A00E00020019900904118029809180498401A0490E0031B
:2020600006D421461A9B199A049800F0B3F94519002706E003A81A9AC05D199990476D1C86
:202080007F1C02988742F5DBE0030CD521461A9B199A049800F09EF9451904E01A9A302076
:2020A000199990476D1C0099481E00900029F5DC08E00D980D990078491C0D911A9A199971
:2020C00090476D1C0199481E01900029F1DC63E109280100303132333435363738396162D3
:2020E0006364656600000000303132333435363738394142434445460000000000F05AF969
:202100004519761C3078002800D0E2E528461BB0F0BD600700D406271898C01DC108C900FB
:2021200048680A680831C30FDB071891190001D09CA108E0210501D59BA104E0E10701D003
:202140009AA100E09AA1430011985B08109165280CD006DC452809D046281DD0472841D1CC
:2021600041E0662818D067283CD13CE00021112F01DB112000E0781C0191009008A911A8A2
:20218000FFF7E8FC139905910021119A15927F1C12980197009150E00120C0070390012076
:2021A000019008A9009711A8FFF7D4FC139A149905920022119B009212981593059A0192F2
:2021C000002901D0104602E0791C40180190381A01D5019804E04042401E0090781C019015
:2021E000C01B029043E0012F00DA01270021112F01DD112000E038460191009008A911A8C3
:20220000FFF7A8FC13990591119A0021129815920091019721070CD40599B94201DB019985
:2022200000E00191012904DD159A491E515C302906D0B84201DA011D05DA0121029115E0B3
:202240000199491EEDE7002805DC0099411800910199091A03E0019A411C914200DD019143
:202260000099401A401C02900120C0070390200706D402990198814202DB0020C043029078
:2022800000206946C87707AF012103980337C907884224D0022011902B2012900398002882
:2022A0000CDA404203902D20129007E00A210398FDF722FF30317F1E039039701199481E28
:2022C00011900029F2DC03980028EFD1791E129808703078202108404530BF1E387006A851
:2022E000C01BC01D039010980078002800D00120019941180298C01709180398091804987D
:20230000401A401E0490E00306D421461A9B199A049800F05FF8451910980078002803D089
:202320001A9A199990476D1CE00324D521461A9B199A049800F04EF845191CE00098002840
:2023400007DB00990598884203DD1598405C199901E0199930201A9A904700986D1C401CD5
:2023600000900298401E0290002804D11A9A2E20199990476D1C0199481E01900029DDDCBF
:2023800005E038781A9A7F1C199990476D1C0399481E03900029F4DC21461A9B199A04984E
:2023A000ACE600002D0000002B0000002000000000000000F8B5044600251E4617468804AA
:2023C00004D405E039462020B0476D1C641EF9D52846F8BDFFB50446002581B01E46C8030B
:2023E00001D5302700E02027880404D505E038460399B0476D1C641EF9D5284605B0F0BD85
:202400000A68531C0B6010707047000070B5EFF31080C007C4170120641C444072B60D4D59
:202420006868002800D12C706868401C04D1332209490AA000F02AFB6868002806D0002CD6
:2024400004D1372204490FA000F020FB6868401C686070BDFC000020D8340008696E746546
:2024600072727570745F656E61626C655F636F756E746572203C2055494E5433325F4D41EC
:2024800058000000696E74657272757074735F64697361626C65640010B50E4C60680028DE
:2024A00016D0EFF31080C007C0170121401C484004D14822084909A000F0E8FA6068401EEF
:2024C00060606068002803D12078002800D162B610BD0000FC000020D8340008696E746522
:2024E0007272757074735F64697361626C65640000487047AC32000870B504460020205EA3
:202500000D46401C04D14722064907A000F0BEFA0B48012D205E03D0002100F017FB70BD0E
:202520000121FAE7003300086F626A2D3E70696E20213D202850696E4E616D65294E430048
:202540000000000070B5064601800C46481C14D02006000FFEF782FE05460021204600F083
:20256000F5FA2107090F01208840706028461030B060083028353561F06070BD70B50026C2
:2025800005460C46FFF7DEFF611C07D000212846FFF7B2FF3146284600F052F870BD0000F5
:2025A00070B50D4604460026FFF7CCFF6D1C12D0A05F401C04D135220749084800F066FA90
:2025C00021696068086001212046FFF795FF3146204600F035F870BD643400082826000812
:2025E000F8B504460E4600271546FFF7ABFF761C16D0E05F401C04D135220A490AA000F042
:2026000045FA6068002D01D0E16800E02169086001212046FFF770FF3946204600F010F8D0
:20262000F8BD0000643400086F626A2D3E70696E20213D202850696E4E616D65294E430030
:2026400010B502460020105E00F0B6FA10BD000070B505461D480C4681420AD08000844268
:2026600007D01B48844204D070221A491AA000F00DFA264B28680121C90318608269120478
:2026800001D5491EFAD22248201819D02149401819D04900C84201D11F4858600120D8605E
:2026A00000201861D86118629860586198611748FEF700F9002802D018A0C046C04670BDEC
:2026C0001C485860EAE71C48E7E70000A086010040420F005833000828687A203D3D20319B
:2026E000303030303029207C7C2028687A203D3D2034303030303029207C7C2028687A2016
:202700003D3D20313030303030302900740100206079FEFF206CFBFF0E04300043616E6EF2
:202720006F7420696E697469616C697A6520493243000000382960202A12B000F7B50546C2
:202740002A49019800F07CFA04462949029800F077FA0146204600F059FA2860401C04D1A7
:202760003F22244924A000F091F9294F01262868284C7605B84220D12748016800291CD156
:20278000012101602548C16803221203914382148918C160A06B3043A0631449019800F053
:2027A0007DFA1349029800F079FA0321019800F003FA0321029800F0FFF919490120096805
:2027C000C0038A69120401D5401EFAD22868B84205D1A06A3043A062A06AB043A0621149F5
:2027E0002846FFF735FF03B0F0BD00003831000868310008583300086F626A2D3E69326398
:2028000020213D20284932434E616D65294E43000054004000100240D4000020401002408D
:2028200074010020A086010010B4006881680123DB0399438160816889B28C0A1106A40291
:20284000490E49002143816081681943816010BC704702689068012980B203D04004400CC9
:20286000906070470121C9030843F9E701680A4801608A690020D24312040CD48A69D24356
:20288000120708D48869C043C00301D4012000E003200822CA61704774010020F0B4944674
:2028A00007460E4A3B68002013600C4B0E5C1D683A68AB69DB439B0708D5094CAB69DB431D
:2028C0009B0703D5641E631CF8D100E09662401CC0B26045E9DBF0BC7047000074010020AD
:2028E000FF0F000010B50146406870225043174A002380180A6802608A684260CA68826059
:202900000A69C2604A6902614A690261CA6982610246403253821382538313831A228A5E2C
:20292000521C0DD018228A5E521C0CD00C214161FEF7FEFB002802D005A0C046C04610BDAB
:2029400008214161F4E70421F1E70000C401002043616E6E6F7420696E697469616C697A9F
:202960006520554152540A0084B03C48FFF72DF83B4C0020205E401C04D1352239493AA0B0
:2029800000F084F821696068086010213C48FFF761F805243B4D24073948FFF764F8012835
:2029A000FAD028786946087001223548FFF748F82B4E0020305E401C04D1352229492AA0C5
:2029C00000F064F8F168706808600A2000F0A8FB234E0020305E401C04D13522214922A082
:2029E00000F054F83169706808601C48FEF7E0FF254E30462169401EC943890601D500281F
:202A0000F8D11648FEF7F1FF07462069761E800601D5002EF9D11148FEF7E7FFC01B0101DB
:202A2000686040186421FDF767FBA8603C280FDB1921490188420EDCC72802DC287A3C382A
:202A400004E0A868CD214843C01278302870A3E73C20A860F2E7A960F3E700002C01002000
:202A600004010020B43200086F626A2D3E70696E20213D202850696E4E616D65294E43002E
:202A8000CC000020C0000020A086010070B514460D460646FFF7BAFC23462A46314603A086
:202AA00000F028F800F01CF870BD00006D626564206173736572746174696F6E2066616920
:202AC0006C65643A2025732C2066696C653A2025732C206C696E65202564200A000000002A
:202AE000FFF794FC962000F00DFB962000F00AFBF8E700000FB470B5A0B025AC249DFFF758
:202B000085FC224629466846FEF7C6FF051E11DD0C480068002804D10F2202210A4800F095
:202B2000E7F800246E46315D074800F06DF9641CAC42F8DBFFF7B0FC20B070BC08BC04B054
:202B400018470000D8000020F4030020F0B5044685B00D46401C04D16022104910A0FFF7DE
:202B600095FF68062F07460F6805050F200624073F0F000F240FFEF771FB0121A140009171
:202B80000C4AB9005158019103210391029604956946FDF7DBFD05B0F0BD0000B03300083A
:202BA00070696E20213D202850696E4E616D65294E4300004032000870B505460C46401C0E
:202BC00004D185220B490CA0FFF760FF28062D07000F2D0FFEF742FB022C00D90024C268F0
:202BE000690003238B409A43C260C2688C402243C26070BDB033000870696E20213D2028DA
:202C000050696E4E616D65294E430000884202D0421C01D10846704710B5491C04D003A0E0
:202C2000C046C0460020C04310BD000070696E6D6170206D69732D6D617463680000000070
:202C4000002210B5D243431C0BD00023CB5E5B1C0ED00023CB5E834205D14C68601C08D0AE
:202C60000AE0104610BD0C23CB5E0C315B1CF0D1144602A0C046C046204610BD70696E6D8B
:202C80006170206E6F7420666F756E6420666F72207065726970686572616C0010B50446F4
:202CA000401C0FD00020085E401C12D00020085EA04208D189682046FFF748FF00212046B9
:202CC000FFF77AFF10BD0C20085E0C31401C0028ECD102A0C046C04610BD0000636F756C7A
:202CE00064206E6F742070696E6F757400000000F8B50E460446154634493046FFF7A0FF12
:202D0000074633492846FFF79BFF01463846FFF77DFF2060401C04D165222E492EA0FFF742
:202D2000B5FE344F21683448B9420CD1826A012149040A438262826A8A438262826B0A431D
:202D40008263012161602D4A216891420CD1826A012189040A438262826A8A438262826BA5
:202D60000A4382630221616018493046FFF796FF17492846FFF792FF701C03D0012130468F
:202D8000FFF71AFF681C03D001212846FFF714FF0020E0604B212061C9016061A160E0611A
:202DA000268320466583FFF79DFD2068B8420BD113490120086013482ECC064644362EC63A
:202DC0002ECC2EC621684166F8BD000098310008EC310008083400086F626A5F732D3E75F9
:202DE00061727420213D2028554152544E616D65294E4300004400400010024000480040F1
:202E0000D8000020B0030020406870225043064A83181868C269D2431206D217521CF9D037
:202E2000C8B2196888627047C4010020054A044911604863C86802221043C86070470000D3
:202E4000000801401804002010B504460068C0688047606840680028206811D04068804717
:202E600061680246486803689A1A002A0BDC82684A60616809680029EBD040688847E8E769
:202E80008068804710BD4868216800680969884710BD006840680047F8B52948416A294C72
:202EA0008EB220600169C943C90709D1C168C943C90705D1891E016123490888401C08806E
:202EC00020680169C94389071ED4C168C94389071AD40221C94301611C4D2888002805D018
:202EE0002888FFF7A3FF002028800DE0184F3868002807D01748FFF799FF2E803868401E36
:202F0000386001E000F054F820680169C943490715D4C168C943490711D40421C9430161C8
:202F20002068456A0C4E30687D27281AFF00B84205D3FDF711FD2168E81988633560F8BDF0
:202F4000000801403C010020E8000020EA000020F0000020FFFF0000D0000020064905481F
:202F600008600169C943890702D40221C943016170470000000801401804002004490348A8
:202F80000860C16802229143C1607047000801401804002005484168002906D110B501216E
:202FA00041600020FDF7F0FC10BD7047E800002010B50248FFF748FF10BD0000AC320008E5
:202FC00030B51A4C83B06068002804D1012060600020FDF7D9FC1748154B174A00680169F2
:202FE000C943890500D4036121886D46A9800169C943C90702D1A988491CA980516A29813D
:20300000218829800169C943C90702D12988491C29802946AD8809888D42E0D16946088892
:2030200009890004084303B030BD0000E8000020FFFDFFFF1804002000080140F0B52C4C6B
:203040000746606883B0002804D1012060600020FDF79AFC284B274D284918680269D24348
:20306000920500D4056122886E46B2800269D243D20702D1B288521CB2804A6A32812288D8
:2030800032800269D243D20702D13288521C32803246B68812889642E0D16A4610881289BC
:2030A000000410434A6A381A92B2002803DCFFF77FFF03B0F0BD0514A5606080104867884F
:2030C000861A0225BE4209D360881960101880B24863C8682843C860002006E019604863FA
:2030E000C8682843C8606088801B608003B0F0BDE8000020FFFDFFFF1804002000080140C3
:20310000FFFF000070B57D21C90048430446FFF757FF0546FFF754FF401BA042FAD370BD39
:2031200070B50546FFF74CFF0446FFF749FF001BA842FAD370BD00000A00000000540040B9
:20314000840000000D0000000054004084010000170000000054004084000000FFFF000098
:20316000FFFFFFFF0000000004000000005400408401000009000000005400408400000015
:20318000160000000054004084000000FFFF0000FFFFFFFF0000000001000000004800407E
:2031A0001303000002000000004400401302000004000000004800401303000009000000B3
:2031C00000440040130200000E000000004400401302000016000000004400401300000002
:2031E000FFFF0000FFFFFFFF000000000000000000440040130000000300000000440040B7
:20320000130200000A00000000440040130200000D00000000480040130300000F0000003C
:203220000044004013020000170000000044004013000000FFFF0000FFFFFFFF000000004D
:203240000000000001000000110000000200000012000000030000000000111000002110F3
:2032600000003110000012100000221000003210000000100000000000000000010203045D
:2032800006070809030406080C101820300000000001020304000000952F0008C12F0008A9
:2032A0007D2F00085D2F00083D30000898320008F40000202F6578747261732F6D626564DE
:2032C0002F5441524745545F4E55434C454F5F4C3031314B342F5441524745545F53544DCE
:2032E0002F5441524745545F53544D33324C302F6770696F5F6F626A6563742E680000005A
:20330000433A5C4A656E6B696E735C776F726B73706163655C6D6265642D322D6275696CAB
:20332000642D6C6962726172795C746172676574735C5441524745545F53544D5C544152F8
:203340004745545F53544D33324C305C6770696F5F6170692E630000433A5C4A656E6B695A
:203360006E735C776F726B73706163655C6D6265642D322D6275696C642D6C696272617208
:20338000795C746172676574735C5441524745545F53544D5C5441524745545F53544D333F
:2033A000324C305C6932635F6170692E63000000433A5C4A656E6B696E735C776F726B739E
:2033C000706163655C6D6265642D322D6275696C642D6C6962726172795C746172676574BF
:2033E000735C5441524745545F53544D5C5441524745545F53544D33324C305C70696E6D7D
:2034000061702E6300000000433A5C4A656E6B696E735C776F726B73706163655C6D6265E4
:20342000642D322D6275696C642D6C6962726172795C746172676574735C544152474554F1
:203440005F53544D5C5441524745545F53544D33324C305C73657269616C5F6170692E63BC
:2034600000000000433A2F4A656E6B696E732F776F726B73706163652F6D6265642D322D7D
:203480006275696C642D6C6962726172792F2E6275696C642F6D6265642F544152474554D0
:2034A0005F4E55434C454F5F4C3031314B342F5441524745545F53544D2F544152474554EC
:2034C0005F53544D33324C302F6770696F5F6F626A6563742E680000433A5C4A656E6B69A4
:2034E0006E735C776F726B73706163655C6D6265642D322D6275696C642D6C696272617287
:20350000795C706C6174666F726D5C6D6265645F637269746963616C2E63000040350008C5
:20352000C000002044000000EA1A000884350008040100204C030000FA1A0008CDE5FFFF5A
:20354000C800000000000000000000000000000000000000000000000000000000000000A3
:20356000000000000048E8010000000000000000000000000000000000000000000000001A
:043580000000000047
:00000001FF
